:020000040000FA
:02000000942842
:08000800FF00030E8301A000BC
:100010000A08A1008A010408A20029288A110A16E8
:10002000C52A8A110A165E288A0182008A0182077F
:10003000403406345B344F3466346D347C340734DA
:100040007F346F3477347C3439345E3479347134AE
:1000500008008A110A1655228A110A120C1E442819
:10006000B0088A110A12031D3F288A110A1652226B
:100070000C128A110A1655228A110A1244288A1172
:100080000A169421720899008A110A128C1E6F2890
:100090003308603C8A110A12031D4F28A314330849
:1000A000563C8A110A12031859282C168A110A166E
:1000B000F4218A110A12981C6228181218168A1143
:1000C0000A126F288A110A12181D6B281A08B80024
:1000D0008A110A126F281A088A110A166D218A11CC
:1000E0000A128C1C8B288C10633037028A110A127A
:1000F00003187E28B70A8A110A128B28B7016330C9
:1001000036028A110A1203188928B60A8A110A12BD
:100110008B28B601B50A2208840021088A00200E27
:100120008300FF0E7F0E0900FF30A500FF30A60000
:10013000FF30A700FF30A8000F30A9008A110A166F
:10014000A120A3102C128A110A16F42127128A1159
:100150000A161B222C128A110A16F4212C168A1157
:100160000A16F42160308A150A12FD271A081A08A7
:100170001A088A110A1652228C160C168A110A16AF
:1001800055220B178A110A163C218B172C128A1143
:100190000A16F421C030B9003908BA00BB01BC010D
:1001A000BD01BE01BF01C001C1010130D400231156
:1001B000A311D6018A150A12C827D901DA01DB0179
:1001C0006430DC008A150A12DD278A150A124F24D2
:1001D0008A150A12CC26AB128A110A16F7212311AE
:1001E0002B168A110A16FA218A110A12861CFF2878
:1001F0008A110A12D71D03298A110A1206298A11A7
:100200000A12D71D06298A110A123A298A110A12DE
:10021000F8265508543C8A110A12031D15298A151F
:100220000A129F258A110A122B295508583C8A1157
:100230000A12031D21298A150A12A5238A110A12FE
:100240002B295508533C8A110A12031D2B29AB1682
:100250008A110A16F7215608033C8A110A12031D57
:1002600034298A110A128C228A150A1209278A1146
:100270000A12F4288A150A12CC262B128A110A16A1
:10028000FA2142308A110A1660208A110A16562075
:100290002311D501580835028A110A12031C552969
:1002A000D8088A110A12031D6B295508523C8A117D
:1002B0000A1203196B295508463C8A110A120319C0
:1002C0006B298A110A12061D6B293A08FF3C8A1114
:1002D0000A12031D6E298A110A12A5298A110A120F
:1002E000571C79290508FF3A3A04BB008A110A1203
:1002F0007C2905083A04BB003B08FF3C8A110A121E
:10030000031985298A110A1230268A150A1209272B
:100310008A110A12F8265608033C8A110A12031D94
:1003200094298A110A128C223508023C8A110A1279
:100330000318A2298A110A12861EA229AB128A1159
:100340000A16F7218A110A124A298A110A12061D71
:10035000BB29580835028A110A120318BB2955080F
:10036000523C8A110A120319BB295508463C8A11CE
:100370000A12031DBE298A150A12D92445308A1192
:100380000A1660208A110A1656208A110A12861C43
:10039000D0298A110A12D71DD4298A110A12822A59
:1003A0008A110A12D71D822A8A110A12861CDF2995
:1003B0008A110A12D71DE6298A110A12E3298A1125
:1003C0000A12D719E6298A110A125A2A8A110A161C
:1003D000B0208A110A16C1206008DD006108DE0025
:1003E0006208DF002B168A110A16FA210C305E0211
:1003F0008A110A12031CFF298A110A120E2A8A1571
:100400000A1209278A110A16C1206008DD00610856
:10041000DE006208DF008A110A12F6298A110A1624
:10042000B0208A110A16C1206008DD006108DE00D4
:100430006208DF002B128A110A16FA210C305E02C4
:100440008A110A12031C272A8A110A12362A8A15CF
:100450000A1209278A110A16C1206008DD00610806
:10046000DE006208DF008A110A121E2A8A110A12AF
:10047000F8265508543C8A110A12031D452A8A158C
:100480000A129F258A110A124E2A5508583C8A11D1
:100490000A12031D4E2A8A150A12A5235608033C88
:1004A0008A110A12031D572A8A110A128C228A11F4
:1004B0000A12D4292B128A110A16FA218A110A1655
:1004C000B0208A110A16C1206008DD006108DE0034
:1004D0006208DF0046305E028A110A12031C732A8A
:1004E0008A110A12822A8A150A1209278A110A1603
:1004F000C1206008DD006108DE006208DF008A11AB
:100500000A126A2AAB128A110A16F7218A110A12F4
:10051000EF288A110A12892AD60153308A110A1645
:10052000602065308A110A16602074308A110A161C
:10053000602075308A110A16602070308A110A1600
:1005400060208A110A1656200130BC000230BD001E
:100550000330BE000430BF000530C0000630C100CB
:10056000D5012B128A110A16FA215508583C8A1116
:100570000A12031DBE2A8A110A12242E8A150A1293
:1005800009278A110A1690208A110A12A31E0B2E1F
:100590008A110A1678206808D5005508463C8A1149
:1005A0000A12031D082B8A110A1678206808D50044
:1005B0005508313C8A110A12031DE52A57148A1581
:1005C0000A12B7278A110A12EF2A5508303C8A11FD
:1005D0000A12031DEF2A57108A150A12B727463050
:1005E0008A110A1660208A110A12571CFE2A31301D
:1005F0008A110A1660208A110A12022B30308A11E1
:100600000A1660208A110A1656208A110A120B2E29
:1006100055084C3C8A110A12031DC82B8A110A1670
:1006200078206808D50055083F3C8A110A12031D3E
:10063000292B4C308A110A1660200E30E50039084B
:10064000FF3AE60030308A110A16EE208A110A12AB
:10065000C22B8A110A1678206808D5008A110A165A
:1006600078206808D5005508313C8A110A12031D0C
:100670003D2BB9128A110A12442B5508303C8A11BD
:100680000A12031D442BB9168A110A16782068082D
:10069000D5005508313C8A110A12031D532B39121B
:1006A0008A110A125A2B5508303C8A110A12031D6E
:1006B0005A2B39168A110A1678206808D500550871
:1006C000313C8A110A12031D692BB9118A110A12D1
:1006D000702B5508303C8A110A12031D702BB91576
:1006E0008A110A1678206808D5005508313C8A110D
:1006F0000A12031D7F2B39118A110A12862B550805
:10070000303C8A110A12031D862B39158A110A16EC
:1007100078206808D5005508313C8A110A12031D5B
:10072000952BB9108A110A129C2B5508303C8A115E
:100730000A12031D9C2BB9148A110A167820680826
:10074000D5005508313C8A110A12031DAB2B391014
:100750008A110A12B22B5508303C8A110A12031D65
:10076000B22B39144C308A110A1660200E30E50085
:100770003908FF3AE60030308A110A16EE208A1551
:100780000A12B7278A110A1656208A110A120B2E4E
:100790005508543C8A110A12031D9B2C8A110A1613
:1007A00078206808D50055083F3C8A110A12031DBD
:1007B0001A2C54308A110A1660205808EE00643052
:1007C000EF008A110A169722E1006108EF000A3053
:1007D000F0008A110A168022E0006008303E8A117B
:1007E0000A1660205808EE000A30EF008A110A1637
:1007F0009722E3006308EF000A30F0008A110A161E
:100800008022E2006208303E8A110A1660205808F1
:10081000EF000A30F0008A110A168022E400640812
:10082000303E8A110A1660208A110A1656208A1153
:100830000A12982C30305502EF000A30F0008A116D
:100840000A168022E1006108E4006430E5008A11A4
:100850000A16B022E0006008D8008A110A16782033
:100860006808D50030305502EF000A30F0008A11D8
:100870000A168022E3006308E4000A30E5008A11CA
:100880000A16B022E20062085807D8008A110A1638
:1008900078206808D50030305502EF000A30F000AB
:1008A0008A110A168022E40064085807D8008A15C5
:1008B0000A12B72754308A110A1660205808EE0031
:1008C0006430EF008A110A169722E6006608EF00EE
:1008D0000A30F0008A110A168022E5006508303ED1
:1008E0008A110A1660205808EE000A30EF008A11BB
:1008F0000A169722E8006808EF000A30F0008A1113
:100900000A168022E7006708303E8A110A16602026
:100910005808EF000A30F0008A110A168022E90018
:100920006908303E8A110A1660208A110A1656207C
:100930008A110A120B2E5508533C8A110A12031D04
:10094000D62C8A110A1678206808D5005508313C43
:100950008A110A12031DB32C57158A150A12B727DC
:100960008A110A12BD2C5508303C8A110A12031D47
:10097000BD2C57118A150A12B72753308A110A164F
:1009800060208A110A12571DCC2C31308A110A16A8
:1009900060208A110A12D02C30308A110A16602089
:1009A0008A110A1656208A110A120B2E5508443C49
:1009B0008A110A12031D112D8A110A16782068085F
:1009C000D5005508313C8A110A12031DEE2CD714AC
:1009D0008A150A12B7278A110A12F82C5508303CDA
:1009E0008A110A12031DF82CD7108A150A12B7278C
:1009F00044308A110A1660208A110A12D71C072D6A
:100A000031308A110A1660208A110A120B2D3030FB
:100A10008A110A1660208A110A1656208A110A12B3
:100A20000B2E5508473C8A110A12031D4C2D8A11C2
:100A30000A1678206808D5005508313C8A110A1238
:100A4000031D292DD7158A150A12B7278A110A12F4
:100A5000332D5508303C8A110A12031D332DD7114E
:100A60008A150A12B72747308A110A1660208A11A0
:100A70000A12D71D422D31308A110A1660208A11C0
:100A80000A12462D30308A110A1660208A110A1681
:100A900056208A110A120B2E55084D3C8A110A1253
:100AA0000319582D55086D3C8A110A12031D5F2D3C
:100AB0008A150A121323D5018A110A120B2E550822
:100AC0003F3C8A110A12031D0B2E46308A110A166A
:100AD00060208A110A12571C742D31308A110A16AF
:100AE00060208A110A12782D30308A110A1660208F
:100AF0008A110A16562054308A110A1660205808A6
:100B0000EE006430EF008A110A169722E1006108B6
:100B1000EF000A30F0008A110A168022E000600817
:100B2000303E8A110A1660205808EE000A30EF00A5
:100B30008A110A169722E3006308EF000A30F000DA
:100B40008A110A168022E2006208303E8A110A16D3
:100B500060205808EF000A30F0008A110A1680223F
:100B6000E4006408303E8A110A1660208A110A16D1
:100B7000562053308A110A1660208A110A12571D16
:100B8000C82D31308A110A1660208A110A12CC2D24
:100B900030308A110A1660208A110A165620443015
:100BA0008A110A1660208A110A12D71CDE2D3130F4
:100BB0008A110A1660208A110A12E22D30308A1139
:100BC0000A1660208A110A16562047308A110A1622
:100BD00060208A110A12D71DF42D31308A110A16AD
:100BE00060208A110A12F82D30308A110A1660200E
:100BF0008A110A1656204C308A110A1660200E30CF
:100C0000E5003908FF3AE60030308A110A16EE2076
:100C10008A110A1656203608083C8A110A1203184F
:100C2000212E8A110A12061A1C2E2B168A110A1658
:100C3000FA218A110A12202E2B128A110A16FA2181
:100C4000B6018A110A12B52A2B168A110A16FA2140
:100C50008A150A12CC26D501D6018A150A124F2C04
:100C60008A110A12A31D3F2E0E30E5003B08E60054
:100C700030308A110A16EE208A110A1656208A117F
:100C80000A16C1206008DD006108DE006208DF008E
:100C90008A110A123B18652E3A145408BC005D08EC
:100CA000C2005E08C3005F08C40031308A110A1612
:100CB000602020308A110A1660205D08E0005E087E
:100CC000E1005F088A150A1218268A110A12BB1859
:100CD000822EBA145408BD005D08C5005E08C60027
:100CE0005F08C70032308A110A16602020308A114E
:100CF0000A1660205D08E0005E08E1005F088A15C2
:100D00000A1218268A110A123B199F2E3A15540806
:100D1000BE005D08C8005E08C9005F08CA00333025
:100D20008A110A16602020308A110A1660205D0898
:100D3000E0005E08E1005F088A150A1218268A1191
:100D40000A12BB19BC2EBA155408BF005D08CB00AF
:100D50005E08CC005F08CD0034308A110A1660208E
:100D600020308A110A1660205D08E0005E08E1006C
:100D70005F088A150A1218268A110A123B1AD92E00
:100D80003A165408C0005D08CE005E08CF005F0828
:100D9000D00035308A110A16602020308A110A16D8
:100DA00060205D08E0005E08E1005F088A150A1215
:100DB00018268A110A12BB1AF62EBA165408C10058
:100DC0005D08D1005E08D2005F08D30036308A117A
:100DD0000A16602020308A110A1660205D08E000A3
:100DE0005E08E1005F088A150A121826D40A080076
:100DF0008A110A1690208A150A12A31E89288A11C0
:100E00000A1678206808D50055087A3C8A110A121B
:100E1000031D142FD6088A110A12031D142F013046
:100E2000D6008A110A12372F5508613C8A110A121E
:100E3000031D252F5608013C8A110A12031D252F78
:100E40000230D6008A110A12372F5508703C8A11D9
:100E50000A12031D362F5608023C8A110A12031D7E
:100E6000362F0330D6008A110A12372FD6015508C3
:100E7000523C8A110A120319432F5508723C8A11F9
:100E80000A12031D4B2F5230D5008A150A12CC26A8
:100E90008A150A1286285508443C8A110A12031939
:100EA000572F5508643C8A110A12031D922F4430B3
:100EB0008A110A16602065308A110A166020623095
:100EC0008A110A16602075308A110A166020673070
:100ED0008A110A16602020308A110A1660208A11B1
:100EE0000A12A31D832FA3114F308A110A16602006
:100EF00066308A110A16602066308A110A16602050
:100F00008A110A128C2FA3154F308A110A166020FD
:100F10006E308A110A1660208A110A1656208A1528
:100F20000A1286285508433C8A110A1203199E2F7B
:100F30005508633C8A110A12031DC22F47308A11DB
:100F40000A1660208A110A12861CAD2F8A110A1215
:100F5000D71DB12F8A110A12B82F8A110A12D71D74
:100F6000B82F6F308A110A1660208A110A12BC2F1E
:100F700063308A110A1660208A110A1656208A15D3
:100F80000A1286285508543C8A110A120319CE2FDA
:100F90005508743C8A110A12031DD32F5430D50012
:100FA0008A150A1286285508463C8A110A12031926
:100FB000DF2F5508663C8A110A12031DE52F231501
:100FC0004630D5008A150A1286285508533C8A11E6
:100FD0000A120319F12F5508733C8A110A12031DD6
:100FE000F62F5330D5008A150A1286285508563C2C
:100FF0008A150A12031902285508763C8A150A1226
:10100000031D0A288A150A124F245630D5008A1566
:101010000A1286285508583C8A150A120319162800
:101020005508783C8A150A12031D1D288A150A12D4
:10103000A523D5018A150A12862855084E3C8A1523
:101040000A120319292855086E3C8A150A12031D35
:1010500030288A150A12EE21D5018A150A1286282F
:1010600055084D3C8A150A1203193C2855086D3C59
:101070008A150A12031D43288A150A121323D50163
:101080008A150A1286285508493C8A150A1203193E
:101090004F285508693C8A150A12031D58288A15DD
:1010A0000A128B208A150A12CC268A150A12862863
:1010B000203055028A150A12031C642855087E3C0C
:1010C0008A150A1203187A288A150A12A31D77288E
:1010D0000E30E6005508E70030308A110A16D62097
:1010E0003F308A110A1660208A110A1656208A1586
:1010F0000A12862855088A110A1660203F308A1184
:101100000A1660208A110A165620D5018A150A127D
:101110008A28D50108000130E00044308A110A16FF
:10112000602069308A110A16602073308A110A160D
:10113000602070308A110A1660206C308A110A16FD
:10114000602061308A110A16602079308A110A16EF
:10115000602020308A110A16602043308A110A1656
:10116000602068308A110A16602065308A110A16DC
:10117000602063308A110A1660206B308A110A16CB
:1011800060208A110A165620BC01BD01BE01BF01B4
:10119000C001C101D501B6015508723C8A150A1279
:1011A0000319DE285508583C8A150A120319DE284F
:1011B0005508783C8A150A12031DE1288A150A127F
:1011C000E3298A150A12092736082D3C8A150A12C6
:1011D000031895296008013C8A150A12031DF72897
:1011E0000130BC000230E0008A150A129429600820
:1011F000023C8A150A12031D04290230BD00033087
:10120000E0008A150A1294296008033C8A150A1224
:10121000031D11290330BE000430E0008A150A12B4
:1012200094296008043C8A150A12031D1E29043003
:10123000BF000530E0008A150A1294296008053CB9
:101240008A150A12031D2B290530C0000630E00064
:101250008A150A1294296008063C8A150A12031D91
:1012600038290630C1000730E0008A150A12942997
:101270006008073C8A150A12031D4429BC01083086
:10128000E0008A150A1294296008083C8A150A129F
:10129000031D5029BD010930E0008A150A12942966
:1012A0006008093C8A150A12031D5C29BE010A3038
:1012B000E0008A150A12942960080A3C8A150A126D
:1012C000031D6829BF010B30E0008A150A1294291A
:1012D00060080B3C8A150A12031D7429C0010C30EA
:1012E000E0008A150A12942960080C3C8A150A123B
:1012F000031D8029C1010D30E0008A150A129429CE
:10130000BC0ABD0ABE0ABF0AC00AC10A4108093C9C
:101310008A150A1203189429BC01BD01BE01BF0140
:10132000C001C1010130E000B6018A110A16902007
:101330008A150A12A31EE0298A110A167820680865
:10134000D5005508733C8A150A12031DC229533073
:101350008A110A1660208A150A12571DB7295711DB
:1013600030308A110A1660208A150A12BC295715D6
:1013700031308A110A1660208A110A1656208A1501
:101380000A12E0295508643C8A150A12031DE02957
:1013900044308A110A1660208A150A12D71CD829EF
:1013A000D71030308A110A1660208A150A12DD29FA
:1013B000D71431308A110A1660208A110A16562075
:1013C0008A150A12CC288A150A12B7278A150A121A
:1013D000B5268A150A12CC26D50108008A110A16EC
:1013E000522209309F008A110A16552253308A1161
:1013F0000A16602065308A110A1660206E308A1144
:101400000A16602073308A110A1660206F308A1124
:101410000A16602072308A110A16602020308A1164
:101420000A16602041308A110A1660206E308A1137
:101430000A16602061308A110A1660206C308A1109
:101440000A16602079308A110A16602073308A11DA
:101450000A16602069308A110A16602073308A11DA
:101460000A1660208A110A165620D5018A150A121A
:10147000A6275508723C8A150A120319452A5508F1
:10148000783C8A150A12031D482A8A150A12012B74
:101490008A150A12092700308A150A127723E000FC
:1014A0000E30E6006008E70030308A110A16D620B8
:1014B00020308A110A1660206008ED000530EE0029
:1014C0008A110A165822E10061080739BC00013070
:1014D0008A150A127723E0000E30E6006008E70064
:1014E00030308A110A16D62020308A110A16602060
:1014F0006008ED000530EE008A110A165822E2005D
:1015000062080739BD0002308A150A127723E0000D
:101510000E30E6006008E70030308A110A16D62047
:1015200020308A110A1660206008ED000530EE00B8
:101530008A110A165822E30063080739BE000330F7
:101540008A150A127723E0000E30E6006008E700F3
:1015500030308A110A16D62020308A110A166020EF
:101560006008ED000530EE008A110A165822E400EA
:1015700064080739BF0004308A150A127723E00097
:101580000E30E6006008E70030308A110A16D620D7
:1015900020308A110A1660206008ED000530EE0048
:1015A0008A110A165822E50065080739C00005307F
:1015B0008A150A127723E0000E30E6006008E70083
:1015C00030308A110A16D6208A110A165620600871
:1015D000ED000530EE008A110A165822E600660872
:1015E0000739C1008A110A1690208A150A12A31E13
:1015F000FE2A8A110A1678206808D5008A150A1270
:10160000392A8A110A16522206309F008A110A16B8
:1016100055228A150A12A327D5018A150A12CC264B
:101620008A150A12B52E8A110A16522209309F0015
:101630008A110A165522D50100308A150A1277231D
:10164000E0000E30E6006008E70030308A110A162C
:10165000D62001308A150A127723E0000E30E6000A
:101660006008E70030308A110A16D62002308A1549
:101670000A127723E0000E30E6006008E700303001
:101680008A110A16D62003308A150A127723E00041
:101690000E30E6006008E70030308A110A16D620C6
:1016A00004308A150A127723E0000E30E600600845
:1016B000E70030308A110A16D62005308A150A1242
:1016C0007723E0000E30E6006008E70030308A1132
:1016D0000A16D6208A110A1656208A110A16522294
:1016E00006309F008A110A165522D5010800E6002F
:1016F0009F018A110A16522209309F009F1303107E
:101700008A110A16552266080739E8000330E900F5
:101710008A110A166C22E700670880389F001F14A0
:1017200014308A110A16BB211F158A150A121F19B7
:101730009C2B8A150A12A22B8A150A1209278A15D0
:101740000A12952B9F011E08080053308A110A16B1
:10175000602065308A110A1660206E308A110A16E0
:10176000602073308A110A1660206F308A110A16C1
:10177000602072308A110A16602020308A110A1601
:10178000602054308A110A16602065308A110A16CA
:10179000602073308A110A16602074308A110A168C
:1017A00060208A110A165620D5015508723C8A1508
:1017B0000A120319E12B5508783C8A150A12031DF9
:1017C000E42B8A150A12482C0508BB003B083A0690
:1017D000003C8A150A120319342C0E30E5003B0830
:1017E000E60030308A110A16EE208A110A165620B9
:1017F0008A150A123B1C012C0130BC008A150A1202
:10180000022CBC018A150A12BB1C0B2C0230BD0035
:101810008A150A120C2CBD018A150A123B1D152CC3
:101820000330BE008A150A12162CBE018A150A1250
:10183000BB1D1F2C0430BF008A150A12202CBF01CB
:101840008A150A123B1E292C0530C0008A150A127F
:101850002A2CC0018A150A12BB1E332C0630C10087
:101860008A150A12342CC1018A150A1209273B086D
:10187000BA008A110A1690208A150A12A31E452C56
:101880008A110A1678206808D5008A150A12D52B05
:10189000D5018A150A12CC268A150A12B52E5030A7
:1018A0008A110A16602069308A110A1660206E308B
:1018B0008A110A16602065308A110A166020773076
:1018C0008A110A1660206F308A110A1660206F3064
:1018D0008A110A16602064308A110A1660202030AE
:1018E0008A110A16602054308A110A166020693065
:1018F0008A110A1660206D308A110A166020653040
:101900008A110A16602072308A110A16602020306F
:101910008A110A16602076308A110A16602031304A
:101920008A110A1660202E308A110A166020323081
:101930008A110A16602036308A110A1660208A1130
:101940000A16562062308A110A16602079308A11F0
:101950000A16602020308A110A16602042308A114F
:101960000A16602065308A110A16602072308A11CA
:101970000A16602074308A110A16602020308A11FD
:101980000A16602044308A110A16602072308A11CB
:101990000A16602061308A110A1660206B308A11A5
:1019A0000A16602065308A110A1660208A110A160C
:1019B00056288A150A12A31D082D46308A110A16C8
:1019C00060206F308A110A16602072308A110A1660
:1019D000602063308A110A16602065308A110A1669
:1019E000602064308A110A16602020308A110A169D
:1019F000602045308A110A1660206E308A110A165E
:101A0000602064308A110A1660208A110A16562056
:101A1000BC088A150A12031D212D8A150A123918CD
:101A2000212D31308A110A16602020308A110A16C1
:101A300060204208E0004308E10044088A150A12C9
:101A40001826BD088A150A12031D3A2D8A150A1296
:101A5000B9183A2D32308A110A16602020308A11C6
:101A60000A1660204508E0004608E10047088A158C
:101A70000A121826BE088A150A12031D532D8A154C
:101A80000A123919532D33308A110A16602020307A
:101A90008A110A1660204808E0004908E1004A0857
:101AA0008A150A121826BF088A150A12031D6C2D02
:101AB0008A150A12B9196C2D34308A110A16602061
:101AC00020308A110A1660204B08E0004C08E10023
:101AD0004D088A150A121826C0088A150A12031D15
:101AE000852D8A150A12391A852D35308A110A1664
:101AF000602020308A110A1660204E08E0004F084E
:101B0000E10050088A150A121826C1088A150A121F
:101B1000031D9E2D8A150A12B91A9E2D36308A1180
:101B20000A16602020308A110A1660205108E00051
:101B30005208E10053088A150A12182608008A156F
:101B40000A123918B32D31308A110A16602020305C
:101B50008A110A1660204208E0004308E1004408A8
:101B60008A150A1218268A150A12B918C72D32309A
:101B70008A110A16602020308A110A166020450852
:101B8000E0004608E10047088A150A1218268A155F
:101B90000A123919DB2D33308A110A1660202030E1
:101BA0008A110A1660204808E0004908E1004A0846
:101BB0008A150A1218268A150A12B919EF2D34301F
:101BC0008A110A16602020308A110A1660204B08FC
:101BD000E0004C08E1004D088A150A1218268A1503
:101BE0000A12391A032E35308A110A166020203065
:101BF0008A110A1660204E08E0004F08E1005008E4
:101C00008A150A1218268A150A12B91A172E3630A2
:101C10008A110A16602020308A110A1660205108A5
:101C2000E0005208E10053088A150A12182608003D
:101C3000E2006008E3006308EE006430EF008A1100
:101C40000A169722E5006508E4006408003C8A153E
:101C50000A120318302E6408303E8A110A166020DA
:101C60006308EF006430F0008A110A168022E60053
:101C70006608E3006308EE000A30EF008A110A16D6
:101C80009722E7006708E4006408003C8A150A12FE
:101C900003184F2E6408303E8A110A16602063082C
:101CA000EF000A30F0008A110A168022E800680866
:101CB000E4006408303E8A110A1660202E308A1132
:101CC0000A1660206108EF006430F0008A110A16DD
:101CD0008022E9006908E3006308EE000A30EF00A3
:101CE0008A110A169722EA006A08E4006408303E66
:101CF0008A110A1660206308EF000A30F0008A118A
:101D00000A168022EB006B08E4006408303E8A115A
:101D10000A1660206208EF006430F0008A110A168B
:101D20008022EC006C08E3006308EE000A30EF004C
:101D30008A110A169722ED006D08E4006408303E0F
:101D40008A110A1660206308EF000A30F0008A1139
:101D50000A168022EE006E08E4006408303E8A1104
:101D60000A1660208A110A16562852308A110A165D
:101D7000602065308A110A16602061308A110A16C7
:101D8000602064308A110A16602079308A110A16A0
:101D900060208A110A1656283908BA00D6018A111D
:101DA0000A16B0208A150A12A31DED2E52308A1190
:101DB0000A16602065308A110A16602073308A1175
:101DC0000A16602065308A110A16602074308A1164
:101DD0000A1660208A110A165620BC01BD01BE01F8
:101DE000BF01C001C1010130D400C201C301C4015F
:101DF000C501C601C701C801C901CA01CB01CC0197
:101E0000CD01CE01CF01D001D101D201D3012315E3
:101E10000800D90A59085C028A150A120318A22F71
:101E2000D901DA0A5A08063C8A150A1203181A2F31
:101E30000130DA008A150A12D71C252F00308A11CA
:101E40000A1601228A150A12292F3F308A110A1612
:101E500001225A08013C8A150A12031D3B2F3C0837
:101E60008A150A12A8278A110A16FD213E30DB00C6
:101E70008A150A12922F5A08023C8A150A12031D6B
:101E80004D2F3D088A150A12A8278A110A16FD212E
:101E90003D30DB008A150A12922F5A08033C8A153E
:101EA0000A12031D5F2F3E088A150A12A8278A11FD
:101EB0000A16FD213B30DB008A150A12922F5A08C0
:101EC000043C8A150A12031D712F3F088A150A1255
:101ED000A8278A110A16FD213730DB008A150A125D
:101EE000922F5A08053C8A150A12031D832F4008B9
:101EF0008A150A12A8278A110A16FD212F30DB0045
:101F00008A150A12922F5A08063C8A150A12031DD6
:101F1000922F41088A150A12A8278A110A16FD2154
:101F20001F30DB008A150A12D71C9E2F5B083F3A30
:101F30008A110A1601228A150A12A22F5B088A1139
:101F40000A16012208006430DC000800DC010800E9
:101F5000E80068080F398A110A121620E9008A156C
:101F60000A12571DB52FFF30E90669080800E50180
:101F700058088A110A16C9210130E50057088A114C
:101F80000A16C9210230E50039088A110A16C92942
:101F9000D9018A110A16E6215A08D8000130D90061
:101FA0008A110A16E6215A08D7000230D9008A1190
:101FB0000A16E6215A08B90008008A110A165222A8
:101FC00006309F008A110A16552200308A110A161F
:101FD00005223F308A110A16352206308A110A1668
:101FE0003122C0308A110A162D2200308A110A16B9
:101FF000292200308A110A161E2AB9003908C03C6D
:102000008A110A16031D10288A110A16522240301E
:10201000990018158A110A1655228A110A164328A2
:102020003908603C8A110A16031D22288A110A16F3
:1020300052228130990018158A110A1655228A11E8
:102040000A1643283908183C8A110A16031D342839
:102050008A110A1652228130990018118A110A1623
:1020600055228A110A16432839080C3C8A110A168F
:10207000031D43288A110A165222FF3099001811B5
:102080008A110A1655228A110A16522298168A11A6
:102090000A1655221812181698139817A7138A11A2
:1020A0000A16152227138A110A16182A0D308A11CA
:1020B0000A1660200A308A110A1660282408EF00E8
:1020C000EF003008603C8A110A16031D6A288A1145
:1020D0000A1661288B136F088A110A16A8218A1123
:1020E0000A1652220C168A110A1655228B1708005E
:1020F000B3088A110A16031D80288A110A16782847
:10210000133033028A110A1603188A282C128A11F6
:102110000A16F4218A110A1659216A08E8000800F3
:10212000B3088A110A16031D9C28A3128A110A16E5
:10213000A0288A110A16A028A3168A110A16A02818
:1021400008008A110A165222FA3092008A110A16E1
:1021500055220C3092008A110A16B0200B17080085
:102160008A110A1652228C108A110A165522B501BC
:10217000B601B7018A110A1652228C148A110A1666
:10218000552AE2008A110A1652228C108A110A1668
:1021900055223508E0003608E1003708E2008A11D0
:1021A0000A1652228C148A110A16552AE80066086B
:1021B000E900670E0F39EA0068088A110A160A2139
:1021C0006B08E8006608E90067080F39EA0068084C
:1021D0008A110A160A216B08E8000800E700083097
:1021E000E8006508E9006608ED000730EE008A1196
:1021F0000A165822EC006C08EA0067088A110A16D1
:102200000A216B08E7000310E60D8A110A16E80B95
:10221000F1280800EB00EA088A110A16031D1F299D
:10222000EB088A110A1603191C296B08A400033055
:1022300069078A110A1214208A110A163B290A30EA
:102240006A028A110A16031830296A08303EA4006F
:10225000033069078A110A1214208A110A163929D3
:102260000A306A02413EA400033069078A110A124B
:1022700014203030EB0008008A110A1645218A111B
:102280000A1680211030B40008006F30B100103001
:10229000B2006030B90000308A110A166D218A112F
:1022A0000A16B90B4B296F30B1001030B200B301E0
:1022B000080001303302B30001303202B2003208AC
:1022C0000F3C8A110A16031D67296F30B20083176D
:1022D000320884000008EA000800F100B30A8317FE
:1022E000310884007108800001303102B1003108EA
:1022F0000F3C8A110A16031D7F296F30B1000800B8
:10230000EF30AE009030AF006030B90000308A117D
:102310000A16A8218A110A16B90B8629EF30AE00D9
:102320009030AF00B001080001303002B000013041
:102330002F02AF002F088F3C8A110A16031DA22915
:10234000EF30AF0083172F0884000008F200080068
:10235000F000B00A83172E08840070088000013056
:102360002E02AE002E088F3C8A110A16031DBA29D0
:10237000EF30AE000800E800FE30E900FF30EA0070
:102380008A110A1668086907031C00346A07C42901
:102390000800E600831203136608831203178C00FB
:1023A00003136508831203178D0083168C130C1515
:1023B0008B138B1355308D00AA308D008C148C1824
:1023C000DF290C118B17831203130800DA00831224
:1023D0000313590803178D0083168C130C148312F2
:1023E0000C080313DA0008008A110A160C2A8A1155
:1023F0000A160F2A8A110A160F2AAD008A110A1628
:10240000092AAC008A110A160C2AAA008A110A1697
:10241000122A2D08880008002C08870008002B08C5
:10242000860008002A08850008008A110A16492A31
:102430008A110A16492A8A110A16492ADD005D08FE
:102440000F39DE002908F0395E04A9008A110A1646
:10245000392AA8008A110A16412AA7008A110A16E9
:10246000492AA6008A110A164C2AA5008A110A16C2
:102470004F2A29088A110A16522289008A110A163F
:10248000552A28088A110A16522288008A110A162B
:10249000552A270867000800260866000800250856
:1024A0006500080083160313080083120313080055
:1024B000EE006E08003C8A110A16031C622A8A117B
:1024C0000A166A2A0310ED0C01306E02EE008A1122
:1024D0000A16592A6D080800E9006908003C8A11AB
:1024E0000A16031C762A8A110A167E2A0310E80DA2
:1024F00001306902E9008A110A166D2A680808008D
:10250000F000F0088A110A160319952A70086F0264
:102510008A110A1603188F2A8A110A16952A70083A
:102520006F02EF008A110A16862A6F080800EF0072
:10253000F001EF088A110A160319AE2A6F086E021D
:102540008A110A160318A72A8A110A16AE2A6F08DA
:102550006E02EE00F00A8A110A169E2A7008080020
:10256000E500E6016508003C8A110A16031CBB2A37
:102570008A110A16C32A6408E60701306502E500DD
:102580008A110A16B22A660808000E30A400080054
:02400E00723FFF
:00000001FF
